:100000005EC1000078C1000076C1000074C100002C
:1000100072C1000070C100006EC100006CC1000020
:100020006AC1000068C1000066C100000C941A0D8E
:1000300062C1000060C100005EC100005CC1000040
:100040005AC1000058C1000056C1000054C1000050
:1000500052C1000050C100004EC100004CC1000060
:100060004AC1000048C1000046C1000044C1000070
:1000700042C100001303180323032D033303390384
:100080006603720377037C038B0390039B03B70320
:10009000CA03D003D803DE03E403EE033E045E0488
:1000A000740483042C0533053C0543054D055305B5
:1000B00056055D0556055D0556055D0577057E050A
:1000C00087058E0597059D05A005A705A005A70531
:1000D000A005A705850688068B068E06A906A90633
:1000E000A906A906970691069D06A3069A069406F8
:1000F000A006A606E70D0A0EF50E0A0EF50E510E25
:10010000730EF50EC60ED80E2203690062006D0054
:100110002D00630061007000730065006E007300C5
:1001200065002D007500730062000000220354007A
:100130006F006D00200057006F006E0067002D00FB
:1001400043006F0072006E0061006C006C000000E4
:100150000403090409025400030100A0FA09040081
:1001600000010301010009211101000122250007FE
:1001700005810308000A09040100010300000009C9
:1001800021110100012220000705830308000A094C
:10019000040200010300000009211101000122BE38
:1001A000000705820319000A120110010000002057
:1001B000810402000100010200010600FF0901A103
:1001C000010902150025FF7508950881020903152C
:1001D0000025FF750895089102C005010906A101D7
:1001E00005081901290315002501950375019102E0
:1001F000950175059101050719E029E7150025010D
:10020000950875018102050719002931150025019E
:100210009532750181029501750181010507193338
:10022000299B1500250195697501810295017501CC
:1002300081010507199D29A415002501950875015F
:100240008102050119812983150025019503750196
:100250008102050C19B029B8150025019509750111
:100260008102050C09CD09E209E909EA0A8A010AB5
:1002700092010A94010A21020A23020A24020A2591
:10028000020A27020A2A0215002501950D7501812F
:1002900002950175028101C005010906A1017501E0
:1002A00095088101950175088101950575019101F8
:1002B000950175039101950675088101C00011240F
:1002C0001FBECFEFD4E0DEBFCDBF11E0A0E0B1E0B4
:1002D000E6E4F3E202C005900D92AC35B107D9F720
:1002E00013E0ACE5B1E001C01D92A138B107E1F720
:1002F0008FD00C94A11184CE62C348C380E291E0F8
:100300000E945E1080E191E00E945E1080E091E02A
:100310000E945E10E2EEF0E08081846080830895A8
:1003200080E291E00E94280F80E191E00E94280F76
:1003300080E091E00C94280F80912E0190912F0184
:10034000009729F0019790932F0180932E018091BF
:100350001E0190911F01009729F0019790931F01B2
:1003600080931E0180910E0190910F01009729F05A
:10037000019790930F0180930E012FC30F931F934A
:10038000CF93DF93FC01C901E80121E0E032F207DD
:1003900011F44AD405C021E0E031F20721F4D0D1B4
:1003A00088E090E005C066817781F1D489E190E032
:1003B0009983888380E0DF91CF911F910F910895F9
:1003C000AC01C90121E04032520709F4D6C54051C1
:1003D000514009F41BC1D4C584B7877F84BF88E12D
:1003E0000FB6F89480936000109260000FBE90E00A
:1003F00080E80FB6F89480936100909361000FBE7F
:100400003BD00E949D0A0E94A10A469A0C940B0DB3
:10041000E3DF7894F8D365D7D9D7DDD38FE19EE4B5
:100420000197F1F700C000004DD080918C019091B0
:100430008D01019609F464D6A6D5809178038823AE
:1004400021F080917803853041F4809176038823F0
:1004500021F01DD781110E94B70A80E291E00E942D
:10046000711080E191E00E94711080E091E00E94A3
:1004700071100E940E0FE0CF0E948E0A289A0895F4
:10048000CF93DF9390938D0180938C012898EC019A
:10049000CC0FDD1FCC0FDD1F8D2F0E94970A8C2FF4
:1004A0000E94970A289ADF91CF91089560918C015C
:1004B00080E090E00E948F1160918D0181E090E0DA
:1004C0000C948F11CF93DF9381E090E00E9478111C
:1004D000C82FD0E0DC2FCC2780E090E00E9478117C
:1004E0009E01282BC901DF91CF91CACF292F332735
:1004F00023303105C9F064F42130310581F0223018
:10050000310509F043C084E590E024E531E042C0C4
:1005100021323105F1F02232310541F137C082E15B
:1005200090E028EA31E036C099278130910541F00A
:100530008230910541F0892B49F5E0E5F1E005C0F5
:10054000ECE2F1E002C0E8E0F1E0849190E09F018C
:1005500021C06330D8F4E62FF0E0EE0FFF1FE25C1D
:10056000FE4F2081318189E090E014C0633070F447
:1005700070E0FB01EE0FFF1FE85CFE4F2081318130
:10058000FB01EB5CFE4F808190E004C080E090E0D6
:1005900020E030E0FA01318320830895EF92FF924A
:1005A0000F931F93CF93DF938C0191E0EE24E3949C
:1005B000F12C461720F1A62FB0E0AA0FBB1FAA0FFF
:1005C000BB1F20E030E0E801C90FD11DF901EA0F9F
:1005D000FB1FEF56FE4F808183304CF08881F7017E
:1005E000022E01C0EE0F0A94EAF7E82BE8832F5F92
:1005F0003F4F2430310551F76F5F9F5FDACFDF91B6
:10060000CF911F910F91FF90EF900895DC01EC9135
:100610004E2F50E04D30510508F091C0FA01E65CD4
:10062000FF4F0C94451111968C91809332010895DF
:1006300011962C91119712968C9190E0982F882703
:10064000820F911D1DCF11968C91882309F477C0DC
:10065000E0913301F0913401099411968C91882333
:1006600009F46DC023CF11968C91882309F467C0DB
:1006700047C513964C91139712969C911297119619
:10068000EC918E2F8F73873108F059C0943008F0A9
:1006900056C0E295E695E695E370E150E33040F40C
:1006A000F0E0EE0FFF1FEC5BFE4F2081318102C0B6
:1006B00028E532E0E82FF0E0EE0FFF1FEE0FFF1FFE
:1006C000E90FF11DE20FF31F4083089512968C91FC
:1006D00012971196EC91E83090F5F0E0E05FFC4F56
:1006E0008083089511968C91882349F16FC61196E5
:1006F0008C91882321F187C613968C9113971296BB
:100700009C91129711962C9120938F0190938E01BA
:100710008093900154C111968C91882381F049C235
:1007200011968D919D91AC918093ED019093EE0186
:10073000A093EF01089511968C918111CAC5089577
:10074000CF93DF93DC0188E0FD0111928A95E9F7F0
:10075000E0913201EC934E2F50E0FA013197EB30EB
:10076000F10508F0DAC0E95BFF4F0C94451184E015
:1007700011968C93119798E012969C93129797E19B
:1007800013969C93139714968C93149781E0159667
:100790008C93C3C046E060E0CD0100DF83E005C07C
:1007A0004DE067E0CD01FADE84E080933201B5C010
:1007B00044E16EE0CD01F2DE85E0F7CF47E165E18F
:1007C000CD01ECDE82E0F1CF90918C0180918D0122
:1007D00011969C93119712968C939FC080918701DC
:1007E00090918601282F2295220F220F207C292B01
:1007F00011962C931197C0913001D091310112962E
:10080000492F50E0440F551F440F551F20E030E0A2
:10081000F901E40FF51FEC0FFD1F60816D932F5F51
:100820003F4F24303105A1F79F5F973119F0909326
:10083000860173C0109286018F5F843019F0809317
:10084000870102C01092870180918701813061F099
:1008500040F0823081F0833009F05FC084EB92E099
:1008600005C088E592E002C088E193E090933101F1
:100870008093300152C08CEF91E0F8CF80918501D8
:1008800011968C931197E82FF0E0EE0FFF1FEE0FFB
:10089000FF1FE05FFC4F408151816281738112969E
:1008A0004D935D936D937C9315978F5F823019F014
:1008B0008093850132C0109285012FC0E6E5F1E0FA
:1008C00080E090E022E0280F31910196ED01C80F01
:1008D000D91F3883332321F08630910599F727E01B
:1008E000A20FB11D1C9219C080918F0111968C939B
:1008F000119780918E0112968C931297809190019E
:1009000013968C930AC02091ED013091EE01409135
:10091000EF0111962D933D934C93DF91CF91089564
:1009200090918801811103C091FD05C002C091FF23
:1009300002C092FD10C0292F2170882331F09660EB
:100940009093880181E0822708959D7F9460909321
:100950008801822F089580E008958823A1F0809176
:100960008F018D3028F48B3040F4893020F40895C5
:100970008F3028F0089581E003C082E001C083E059
:100980008093740308951092740308952498259811
:10099000269827982C982D982E982F9810928A0197
:1009A00010928901809188018B7F809388018091CA
:1009B0008F01823019F4249A259A269A0895E6DF49
:1009C00080918F01813029F038F083508C3020F4F1
:1009D0002D9A269A279A2F9A089580918A018F3FFF
:1009E00019F08F5F80938A0180918F01813021F00F
:1009F000C8F083508C30B0F490918A0180918E01C0
:100A0000981302C02E98089580918901882351F08F
:100A100020919001921730F010928A0181508093BA
:100A200089012E9A0895809189018F5F80938901B1
:100A300008951F93CF93DF93162FE0918F014E2FD0
:100A400050E0FA013397EC30F10508F03CC0EC01BE
:100A5000EE5AFF4F0C94451183B185FB882780F92E
:100A600091E0892702C083B180725ADF882359F14F
:100A7000C10FD11D89E30FC083B185FB882780F9A1
:100A800091E0892702C083B180724ADF8823D9F0C0
:100A9000C10FD11D83E58A8316C01D9914C08881BA
:100AA0008E5F888310C01D99FACF0DC083B185FB7E
:100AB000882780F991E0892702C083B18072DF9195
:100AC000CF911F914ACFDF91CF911F910895CF937E
:100AD000DF93E0918F014E2F50E0FA013397EC3015
:100AE000F105D0F5EC01E25AFF4F0C94451183B1AA
:100AF00085FB882780F991E0892702C083B1807245
:100B00000FDF882349F188858260888725C083B1FB
:100B100085FB882780F991E0892702C083B1807224
:100B2000FFDE8823C9F08B8588608B8715C01D99EF
:100B300013C08881826088830FC01D99FACF0CC0D2
:100B400083B185FB882780F991E0892702C083B1B2
:100B50008072DF91CF9101CFDF91CF910895909175
:100B60008F01953028F49330B0F4923021F008953D
:100B70009730B8F0089580FF02C02D9A01C02D98DB
:100B800081FF02C02E9A01C02E9882FF02C02C9ACB
:100B900008952C98089581FF06C080918801816096
:100BA00005C080FDFACF809188018E7F80938801F7
:100BB000089560918F018AE791E00E948F11609102
:100BC0008E018BE791E00E948F11609190018CE77C
:100BD00091E00C948F118AE791E00E9478118F3098
:100BE00018F480938F0102C010928F018BE791E07F
:100BF0000E94781180938E018CE791E00E94781119
:100C00008093900108958CE5E1E9F1E0DF011D9208
:100C10008A95E9F78CE0E0EFF1E0DF011D928A951B
:100C2000E9F71092740308956F927F929F92AF92AA
:100C3000BF92CF92DF92EF92FF920F931F93CF93C9
:100C4000DF93EC01FBD38150833048F4E82FF0E0D0
:100C5000EE0FFF1FE65BFE4F4081518102C048E569
:100C600052E000E010E060E0CC24C394D12CF3E02B
:100C7000BF2EA2E0AA2E99249394A62F20E030E064
:100C8000C80195958795FC01E051FE4F7F01702FBB
:100C90007170663008F064C0F7018081E82FF0E0E1
:100CA000772351F0C9010496360102C0660C771C07
:100CB0008A95E2F7C30107C0C601022E02C0880F61
:100CC000991F0A94E2F78E239F23892B09F441C0D0
:100CD000FA01E20FF31FE081E430D8F180E38E0FD8
:100CE0008330B8F16F5FCE018A0F911DDC0112963F
:100CF000EC938E2F90E0FC01E85DF109E031F10505
:100D000040F5E659FF4F0C9445111092740321C031
:100D1000909274031EC0A09274031BC0B09274031F
:100D200018C088818E5F14C08881805E11C0888160
:100D30008F5F0EC08881805F0BC088818C5F08C088
:100D40008881805C05C08881885F02C08881805866
:100D500088832F5F3F4F2430310511F0A62F99CFA4
:100D60000F5F1F4F4C5F5F4F0731110509F085CFB3
:100D7000CE01DF91CF911F910F91FF90EF90DF9007
:100D8000CF90BF90AF909F907F906F9052CE2F9258
:100D90003F924F925F926F927F928F929F92AF920B
:100DA000BF92CF92DF92EF92FF920F931F93CF9358
:100DB000DF9300D000D0CDB7DEB75C014B013ED34E
:100DC0008150833048F4E82FF0E0EE0FFF1FE65B20
:100DD000FE4F8081918102C088E592E07C01412C28
:100DE000512C66246394712C3324339442E0242ED6
:100DF00000E010E0C20195958795FC01E051FE4F9F
:100E00006F01242D21702983F601808190E02981D2
:100E1000222359F098012C5F3F4FA30102C0440FD9
:100E2000551F2A95E2F79A0107C09301002E02C0D0
:100E3000220F331F0A94E2F782239323892B09F4AC
:100E400073C0F701E00FF11F80818B3D31F188F411
:100E5000833D38F4803D08F067C0833008F464C0F7
:100E60003CC0893DA1F0B0F4883DB9F510927403FF
:100E70005BC0853E38F4823E18F5803E09F1813E24
:100E800081F02BC0853E69F0883ED0F026C03092BC
:100E900074034AC02092740347C053E05093740314
:100EA00043C0F401208130E090E2980F02C03595F4
:100EB00027959A95E2F720FD03C08C83B4DD8C81E1
:100EC000805E930102C0220F331F8A95E2F7C901A9
:100ED000F5019081892B808327C0482F4695469540
:100EE000469550E08770F401E40FF51F218130E052
:100EF000082E02C0359527950A94E2F720FD07C019
:100F00004A835B838C838FDD8C815B814A81FA010C
:100F1000EA0DFB1D930102C0220F331F8A95E2F7F1
:100F2000C9019181892B81830F5F1F4F0430110507
:100F300009F06ACF3FEF431A530A44E0E40EF11C74
:100F400057E14516510409F053CFC5010F900F909A
:100F50000F900F90DF91CF911F910F91FF90EF9025
:100F6000DF90CF90BF90AF909F908F907F906F90C9
:100F70005F904F903F902F90AACDFC018081EFCDE4
:100F8000FC018081ECCD4F925F927F928F929F9275
:100F9000AF92BF92CF92DF92EF92FF920F931F9387
:100FA000CF93DF9300D000D0CDB7DEB78CE0E0EF79
:100FB000F1E0DF011D928A95E9F771E9E72E71E012
:100FC000F72E00E010E0AA24A394E5E0BE2EDD2475
:100FD000D394F8ECCF2E902EE02FE695E695E6958B
:100FE000F0E0E351FE4F808190E0202F277002C097
:100FF000959587952A95E2F780FD65C04698802FE4
:10100000A8D2469A19821A821B821C828A2D8A953E
:10101000F1F74899A9824999AA824A99AB824B99DA
:10102000AC82AE014F5F5F4F2701D70120E030E077
:10103000C8019595879580519E4FE92DE1709E2EB0
:10104000722EFA016191AF01F201662319F06081FD
:10105000615002C060816F5F6083BD018C9087FE2C
:1010600002C01C9204C0F5E0F8150CF4BC92119675
:10107000FB0160816330B4F0FC018080992051F065
:10108000B9016C5F7F4FFD2D01C0FF0F6A95EAF734
:101090006F2F05C06D2D01C0660F7A94EAF768299D
:1010A000FC0160832F5F3F4FFFEF4F1A5F0A243030
:1010B000310531F6469845D2469A0631110519F0A8
:1010C0008C2D8A95F1F70F5F1F4F64E0E60EF11C3F
:1010D0000731110509F07FCF0F900F900F900F90FF
:1010E000DF91CF911F910F91FF90EF90DF90CF9004
:1010F000BF90AF909F908F907F905F904F9008959A
:10110000AF92BF92CF92DF92EF92FF920F931F9315
:10111000CF93DF9348E552E027E1B12CD12C80E05A
:1011200090E0FA01E80FF91F3081313021F03230C0
:1011300019F4D39401C0B39401968430910589F7D2
:1011400021504C5F5F4F2111EACFC0E0D0E00FEF9C
:1011500013E0E12CF12CC8018E199F098230910512
:10116000C0F1EC01D695C795CE0DDF1DCE0188D913
:101170008FE891E00197F1F700C0000070E2C72E00
:1011800002DFCA94E9F721E931E068E572E040E066
:1011900080E090E0F901E80FF91F508153303CF0F6
:1011A000FB01E80FF91F5081543008F04F5F0196A2
:1011B0008430910579F72C5F3F4F6C5F7F4F91E052
:1011C0002D3E390729F74D1510F08E01C4CF7E0151
:1011D000C2CF8E01EE24EA9453E0F52EC12CD12C1F
:1011E00097012C193D0922303105C0F1E901D6954E
:1011F000C795CC0DDD1DCE0143D98FE891E0019755
:10120000F1F700C0000040E2A42EBDDEAA94E9F789
:1012100081E991E068E572E040E020E030E0FC0127
:10122000E20FF31F508153303CF0FB01E20FF31F3C
:101230005081513009F44F5F2F5F3F4F243031050B
:1012400071F704966C5F7F4F21E08D3E920729F77E
:101250004B1510F07E01C4CF6E01C2CFC8018C1BAC
:101260009D0B24E0969587952A95E1F76FE070E055
:10127000FBD78C0F9D1F04D9DF91CF911F910F9148
:10128000FF90EF90DF90CF90BF90AF9098CB28E584
:1012900032E041E951E080E090E0FA01E80FF91F07
:1012A0006081633034F0F901E80FF91F6081643028
:1012B00070F401968430910581F72C5F3F4F4C5FAD
:1012C0005F4F82E0243B380731F780E0089581E0EA
:1012D000089543E050E06DE771E08DEE91E00C94ED
:1012E000801143E050E06DE771E08DEE91E0F0D7C2
:1012F0008091ED018F3F71F48091EE018F3F51F4A9
:101300008091EF018F3F31F41092ED011092EE01C8
:101310001092EF010895AF92BF92CF92DF92EF92B9
:10132000FF920F931F93CF93DF93EB015C012CE5AA
:10133000A20EB11C6C01F4E0CF0ED11C7E018C0119
:101340000F5F1F4FD5D78F3F09F480E0F7018193DE
:101350007F01C8010C151D0591F724960A151B0580
:1013600049F7DF91CF911F910F91FF90EF90DF90A0
:10137000CF90BF90AF900895AF92BF92CF92DF927F
:10138000FF920F931F93CF93DF938C01EB0187E1C3
:10139000F82E6E0184E0C80ED11CC80169915C0171
:1013A0002FEFA21AB20ABBD7C501CC15DD05B1F7E4
:1013B0000C5F1F4FFA9469F7DF91CF911F910F9146
:1013C000FF90DF90CF90BF90AF90089510928B0167
:1013D00048E050E062E771E080E193E079D768E5AA
:1013E00072E082E090E097DF68E173E08EE590E0E4
:1013F00092DF6CEF71E08AEB90E08DDF64EB72E0DE
:1014000086E191E088CF48E050E062E771E080E15A
:1014100093E076D768E572E082E090E0ADDF68E1C6
:1014200073E08EE590E0A8DF6CEF71E08AEB90E06E
:10143000A3DF64EB72E086E191E09ECFEF92FF9232
:101440001F93CF93DF9380917403E0918B01E15060
:10145000E33040F4F0E0EE0FFF1FE05BFE4F408111
:10146000518102C048E552E060E070E090E0C1E0E8
:10147000D0E0FB01F595E795E051FE4FA081B0E08B
:1014800020E030E0162F1170112351F0F90134964D
:101490007E0102C0EE0CFF1CEA95E2F7F70107C0DF
:1014A000FE01022E02C0EE0FFF1F0A94E2F7EA23AC
:1014B000FB23EF2B79F0FA01E20FF31FE081E13D0E
:1014C00031F0E23D31F0E03D29F4916003C09260DB
:1014D00001C094602F5F3F4F24303105A9F66F5F44
:1014E0007F4F4C5F5F4F6731710519F6992371F09B
:1014F000E0E1F3E038E03E0F2191422F42954F703A
:10150000491302C0822F8F703E13F6CF80938B0158
:10151000DF91CF911F91FF90EF900895219A209A2B
:10152000229A84E58CBD8DB581608DBD08958EBDF8
:101530000DB407FEFDCF8EB508953C9A3D9A3E9AB4
:1015400008954598449888E1459A45988150E1F777
:10155000089545984498449A459A4598449890E04F
:10156000981721F0459A45989F5FFACF089584E037
:1015700089BD86E089BD09B400FEFDCF8091D80009
:101580008F7D8093D8008091E00082608093E0009E
:101590008091E00081FDFCCF0895CF92DF92EF9221
:1015A000FF920F931F93CF93DF93EC018B017A018E
:1015B000C9D1811133C0E114F10439F0F701808100
:1015C0009181081B190BC80FD91FC12CD12C0115F3
:1015D000110519F18091E80085FD16C08091E800A1
:1015E0008E778093E8001AD4E114F10449F0F701F2
:1015F00080819181C80ED91ED182C08285E00EC043
:10160000A1D1882321F30AC089918093F100015070
:101610001109FFEFCF1ADF0ADACF80E0DF91CF9117
:101620001F910F91FF90EF90DF90CF900895209140
:101630007F03309180032617370748F06115710545
:1016400039F42091E8002E772093E80001C0B90119
:1016500040E06115710581F1209178032223E9F1C1
:101660002530E9F12091E80023FD35C02091E80004
:1016700022FD2BC02091E80020FFEBCF2091F2004B
:1016800030E0FC01CF016115710559F020323105C0
:1016900040F481918093F100615071092F5F3F4FB9
:1016A000F1CF41E02032310509F040E02091E8001F
:1016B0002E772093E800CDCF4111CECF06C0809188
:1016C0007803882351F0853051F08091E80082FF43
:1016D000F6CF80E0089581E0089582E0089583E0E8
:1016E00008956115710529F42091E8002B77209366
:1016F000E800FC016115710521F1809178038823D0
:1017000041F1853041F18091E80083FD20C0809156
:10171000E80082FFEFCF8091F200882331F08091C2
:10172000F100819361507109B1F78091E8008B77E6
:101730008093E800DFCF80917803882351F08530D3
:1017400051F08091E80080FFF6CF80E0089581E0BD
:10175000089582E0089583E0089520917F033091F9
:1017600080032617370748F06115710539F4209179
:10177000E8002E772093E80001C0B901FC0120E0C9
:101780006115710569F1809178038823D1F1853065
:10179000D1F18091E80083FD32C08091E80082FDA4
:1017A00028C08091E80080FFEBCF8091F20090E0AC
:1017B0006115710559F08032910540F42491209310
:1017C000F1003196615071090196F2CF21E08097C6
:1017D00009F020E08091E8008E778093E800D0CF78
:1017E0002111D1CF06C080917803882351F0853034
:1017F00051F08091E80082FFF6CF80E0089581E00B
:10180000089582E0089583E00895982F953058F563
:101810009093E900981739F07091EC002091ED0059
:101820005091F00003C0242F762F50E021FF19C003
:101830003091EB003E7F3093EB003091ED003D7F27
:101840003093ED003091EB0031603093EB007093FA
:10185000EC002093ED005093F0002091EE0027FF64
:1018600007C09F5FD3CF8F708093E90081E0089518
:1018700080E00895EF92FF920F931F93CF93DF9331
:10188000E62EEC018C010C5F1F4FF12CFE1499F138
:101890009881992359F1F801208169817A813197E2
:1018A0003081892F8F70853010F080E025C0223084
:1018B00010F442E001C046E0E8E0F0E020E0E61786
:1018C000F70720F42F5FEE0FFF1FF9CF2295207F3F
:1018D000422B232F2295220F220F207C991F99271C
:1018E000991F622F692B91DF8823F9F2F3942596D3
:1018F0000B5F1F4FCBCF81E0DF91CF911F910F91F5
:10190000FF90EF9008958091790387FF11C0809137
:10191000E80082FD05C0809178038111F8CF11C0E5
:101920008091E8008B770BC080917803882349F081
:101930008091E80080FFF8CF8091E8008E77809357
:10194000E80008952091E4003091E50095E640918B
:10195000EC00842F817040FF22C08091E80080FD60
:101960001CC080917803882391F0853091F080919C
:10197000EB0085FD10C04091E4005091E500421756
:10198000530729F39A01915011F784E0089582E0FA
:10199000089583E0089581E0089580E008954091DE
:1019A000E80042FFDECF08953FD041D08091D800BB
:1019B0008F778093D8008091D80080688093D8007A
:1019C0008091D8008F7D8093D80084E089BD86E027
:1019D00089BD09B400FEFDCF109278031092750303
:1019E0001092760342E260E080E00FDF8091E10038
:1019F0008E7F8093E1008091E20081608093E2001D
:101A00008091E20088608093E2008091E0008E7F08
:101A10008093E0000895E3E6F0E080818E7F80838C
:101A200081E080937703C0CF1092E2000895109276
:101A3000E10008951F920F920FB60F9211242F9379
:101A40003F934F935F936F937F938F939F93AF9346
:101A5000BF93EF93FF938091E10082FF0BC08091D1
:101A6000E20082FF07C08091E1008B7F8093E1005C
:101A70000E949C018091E10080FF18C08091E200EB
:101A800080FF14C08091E2008E7F8093E2008091FD
:101A9000E20080618093E2008091D80080628093B0
:101AA000D80019BC109278030E947D018091E1005A
:101AB00084FF2EC08091E20084FF2AC084E089BDAB
:101AC00086E089BD09B400FEFDCF8091D8008F7DEE
:101AD0008093D8008091E1008F7E8093E100809117
:101AE000E2008F7E8093E2008091E200816080932B
:101AF000E20080917503811106C08091E30087FDAB
:101B000002C081E001C084E0809378030E947C01E0
:101B10008091E10083FF22C08091E20083FF1EC01C
:101B20008091E100877F8093E10082E080937803D9
:101B3000109275038091E1008E7F8093E100809187
:101B4000E2008E7F8093E2008091E20080618093CA
:101B5000E20042E260E080E058DE5FD1FF91EF9169
:101B6000BF91AF919F918F917F916F915F914F91B5
:101B70003F912F910F900FBE0F901F9018951F93BC
:101B8000CF93DF93CDB7DEB7AA970FB6F894DEBF39
:101B90000FBECDBFE9E7F3E088E08E0F9091F10032
:101BA00091938E13FBCF0E9490018091E80083FFF8
:101BB0001CC18091790390917A03492F50E04A30FB
:101BC000510508F012C1FA01E658FF4F5EC3803894
:101BD00081F0823809F009C180917D038F70809374
:101BE000E9008091EB0085FB882780F91092E900DD
:101BF00007C080917603882311F082E001C080E065
:101C00009091E800977F9093E8008093F100109204
:101C1000F100C7C0282F2D7F09F0E7C0882319F0F5
:101C2000823061F0E2C080917B03813009F0DDC039
:101C3000933009F080E0809376032DC080917B0380
:101C4000811129C080917D038F7009F4CEC08093EB
:101C5000E9009091EB0090FF1EC090917A039330C1
:101C600021F48091EB00806214C09091EB009061B0
:101C70009093EB0021E030E0A90102C0440F551F12
:101C80008A95E2F74093EA001092EA008091EB0017
:101C900088608093EB001092E9008091E800877FD4
:101CA00083C08111A2C010917B031F778091E30054
:101CB0008078812B8093E3008091E800877F809378
:101CC000E80021DE8091E80080FFFCCF8091E300F6
:101CD00080688093E300111102C082E001C083E0BC
:101CE0008093780382C08058823008F07EC0809153
:101CF0007B0390917C038C3D53E0950771F583E065
:101D00008A838AE289834FB7F894DE01139620E034
:101D10003EE051E2E32FF0E050935700E49120FFC2
:101D200003C0E295EF703F5FEF708E2F90E0EA30D6
:101D300010F0C79601C0C0968D939D932F5F2431FC
:101D400049F74FBF8091E800877F8093E8006AE2FF
:101D500070E0CE0101966BDC13C0AE014F5F5F4FA8
:101D600060917D030E947602BC01009709F43DC09A
:101D70009091E800977F9093E80089819A81EDDC4B
:101D80008091E8008B778093E8002FC0803869F558
:101D90008091E800877F8093E800809175038093AD
:101DA000F1008091E8008E778093E800ACDD1DC0E3
:101DB00081111BC090917B039230B8F48091E800B0
:101DC000877F8093E800909375039DDD8091750374
:101DD000811106C08091E30087FD02C081E001C04F
:101DE00084E0809378030E947E018091E80083FF65
:101DF0000AC08091E800877F8093E8008091EB0023
:101E000080628093EB00AA960FB6F894DEBF0FBEF7
:101E1000CDBFDF91CF911F9108950895CF93809109
:101E20007803882399F0C091E900CF709091EC007D
:101E3000892F817090FD80E8C82B1092E900809175
:101E4000E80083FD9CDECF70C093E900CF91089538
:101E50006F927F928F929F92AF92BF92CF92DF92BA
:101E6000EF92FF920F931F93CF93DF9300D01F92B7
:101E7000CDB7DEB77C01CDB6DEB68091E80083FF3A
:101E800006C1F701808190E020917D0330917E03AF
:101E90002817390709F0FBC080917A03833009F4D1
:101EA0009DC030F4813071F0823009F4D4C0EFC0AD
:101EB0008A3009F4B8C08B3009F4A1C0893009F028
:101EC000E6C04EC080917903813A09F0E0C08DB63A
:101ED0009EB61A82198280917B0310917C038B83BA
:101EE000F7018085482F50E08DB79EB7841B950B76
:101EF0000FB6F8949EBF0FBE8DBFEDB7FEB73196FB
:101F00005F0160E070E0CF01DCD14FEF410F8E0147
:101F10000F5F1F4F9501BE016D5F7F4FC7010E948C
:101F2000BE01F70186819781009721F0408550E03E
:101F3000B501BED11092E9008091E800877F8093BF
:101F4000E80069817A81C50172DB8091E8008B77B6
:101F50008093E8000FB6F8949EBE0FBE8DBE97C06A
:101F600080917903813209F092C0ADB6BEB600917E
:101F70007F031091800370907B0360907C038DB78A
:101F80009EB7801B910B0FB6F8949EBF0FBE8DBFFE
:101F9000EDB7FEB731964F018091E800877F8093BF
:101FA000E800B801CF019DDB8091E8008E77809337
:101FB000E80021E0711001C020E030E0021B130BAB
:101FC000280D391D4FEF460D672DC7010E94E00116
:101FD0000FB6F894BEBE0FBEADBE59C08091790356
:101FE000813A09F054C08091E800877F8093E8002F
:101FF0008091E80080FFFCCFF701818540C080918F
:102000007903813209F043C08091E800877F809393
:10201000E80079DC90917B0381E0911101C080E0C0
:10202000F701818734C080917903813281F58091F5
:10203000E800877F8093E80066DC80917B039091C5
:102040007C03882736E0969587953A95E1F7F70166
:10205000958784871CC080917903813AC1F480916F
:10206000E800877F8093E8008091E80080FFFCCF44
:10207000F7018485958596958795969587958093A4
:10208000F1008091E8008E778093E8003CDC0FB689
:10209000F894DEBE0FBECDBE0F900F900F90DF9173
:1020A000CF911F910F91FF90EF90DF90CF90BF9055
:1020B000AF909F908F907F906F900895FC0139961C
:1020C00027E0DF011D922A95E9F721E0FC01218735
:1020D00024EF31E03587248723E0248361E00196F3
:1020E000C9CB4F925F926F927F928F929F92AF92E5
:1020F000BF92CF92DF92EF92FF920F931F93CF93F5
:10210000DF9300D01F92CDB7DEB77C01ADB6BEB66F
:1021100080917803843009F08EC08091E400909122
:10212000E500F701228533852817390709F483C0B4
:1021300081818F708093E9008091E80085FF7BC0EA
:102140008DB69EB6408550E08DB79EB7841B950B2B
:102150000FB6F8949EBF0FBE8DBFEDB7FEB7319698
:102160006F011B821A82198260E070E0CF01A9D052
:102170008E010F5F1F4F960140E0BE016D5F7F4FE4
:10218000C7010E94BE01482EF70184859585892BE1
:1021900051F091E080E026853785232B09F090E00F
:1021A000092F182F02C000E010E0F7016680778049
:1021B0006114710489F049815A81B301C6016BD061
:1021C00055245394892B09F4512CF701408550E094
:1021D000B601C3016DD001C0512C89819A81892B30
:1021E000F1F0411004C0511002C0012BC1F0F70101
:1021F000848595859787868781818F708093E90094
:102200008B8181118093F10069817A8140E050E0F7
:10221000C601C3D98091E8008E778093E800809151
:10222000E4009091E500F701938782870FB6F89458
:102230009EBE0FBE8DBE0FB6F894BEBE0FBEADBE25
:102240000F900F900F90DF91CF911F910F91FF9002
:10225000EF90DF90CF90BF90AF909F908F907F9046
:102260006F905F904F9008950024552704C0080E8A
:10227000591F880F991F009729F076956795B8F335
:102280007105B9F7802D952F0895EE0FFF1F05906A
:10229000F491E02D0994FB01DC0104C08D910190C3
:1022A000801921F441505040C8F7881B990B0895BC
:1022B000FB01DC0102C001900D9241505040D8F763
:1022C0000895DC0101C06D9341505040E0F708953E
:1022D000DC01CB01FC01F999FECF06C0F2BDE1BDE6
:1022E000F89A319600B40D9241505040B8F70895D5
:1022F000F999FECF92BD81BDF89A992780B50895CE
:10230000DC01A40FB51F4150504040F0CB01840FB9
:10231000951F2E9105D041505040D8F70895262F93
:10232000F999FECF92BD81BDF89A019700B40216CB
:1023300039F01FBA20BD0FB6F894FA9AF99A0FBE79
:062340000895F894FFCFA0
:102346000282190000015C01190000000000000073
:10235600018308000001750108000000000000006C
:102366000081080000017D01080000000000000057
:1023760058020200182520BE9802BA01DA01660149
:102386007F0198011803FC01B4021803FC01B40292
:0C2396001803FC01B402302E372E30007A
:00000001FF
